:100000000C942A000C947F031895000018950000AA
:10001000189500001895000018950000189500002C
:100020000C9441010C949603189500000C946B04F9
:10003000189500001895000018950000189500000C
:1000400018950000189500001895000018950000FC
:10005000189500008FE58DBFC0E4E8E34E2E84E0E4
:100060008EBFD4E0F4E05F2EEEEFF3E0A0E6B0E068
:10007000A89584B7082E877F84BF88E1992781BD22
:1000800091BD88278D933197E9F789E189B980E09F
:1000900080BD88E18AB96624579A8FEF8ABB8FEFBB
:1000A0008BBB8FEF87BB8FEF88BB8FEF84BB8FEF4E
:1000B00085BB8AED81BB8FE982BB80E08FBD82E08A
:1000C0008EBD89B7846089BF85B78C7F85BF8BB7AC
:1000D00080648BBF7894E1E0F0E00E94DB03A0E352
:1000E000B0E08C9185FBA2E3B0E08C9186F98C9313
:1000F0000E94A303082F013011F00C941E010E94EE
:10010000A903AFE7B0E08C9300917F000F3718F0A0
:1001100011F00C948D000C94A80080E080937E0078
:1001200080917F008093B10000917F00003811F42E
:100130000C94A30000917F004FE70423A2EBB0E0F2
:100140000C930C94A60080E08093B2000C941E01E6
:10015000AEE7B0E08C918F5F8C9380917F00AEE72B
:10016000B0E0AD90BB24AFE7B0E0AA0DBB1D8C930F
:100170000091B10040917F00040FA1EBB0E00C931F
:1001800000917E00093111F00C941E010091B10024
:1001900040919800041BA1EBB0E00C93A1EBB0E000
:1001A0000C9142E00E9497040C93409198000091BA
:1001B000B100041711F00C941E018EB5887F8EBD1E
:1001C00081E080937E0000917E00083118F011F0EC
:1001D0000C940401AEE7B0E0AD90BB24AFE7B0E013
:1001E000AA0DBB1D8C91AEE7B0E0AD90BB24A8E991
:1001F000B0E0AA0DBB1D8C93AEE7B0E08C918F5F91
:100200008C9310F40C94E30082E08EBD0091B20058
:10021000003011F40C941E018091B2008093B30061
:1002200082E88093B2000091B300023011F00C9488
:100230001E0131E0A2EBB0E00E94D2030027A4EB44
:10024000B0E08C9187FB0EF401E041E0041711F05F
:100250000C943D018091B4008F778093B40000919D
:10026000B800003011F00C943A0131E0A7EBB0E097
:100270000E94D2038BB780648BBF0C946F00F894FC
:10028000FFCF0F921F922F923F924F925F927F92D9
:10029000AF92BF920F931F932F933F934F935F9310
:1002A0006F937F938F939F93AF93BF93CF93DF937E
:1002B000EF93FF938FB78F9386E09FEF9DBD8CBD2B
:1002C000ADE7B0E08C918F5F8C9300917D00043698
:1002D00011F00C946E0180E080937D0040919900B4
:1002E00000917D00041710F00C947D018091BA00FC
:1002F00082608093BA000C9482018091BA008D7F55
:100300008093BA0040919A0000917D00041710F08C
:100310000C9491018091BA0084608093BA000C948F
:1003200096018091BA008B7F8093BA0040919B0028
:1003300000917D00041710F00C94A5018091BA0083
:1003400081608093BA000C94AA018091BA008E7FDC
:100350008093BA0040919C0000917D00041710F03A
:100360000C94B9018091BA0080618093BA000C941A
:10037000BE018091BA008F7E8093BA0040919D00AB
:1003800000917D00041710F00C94CD018091BA000B
:1003900080628093BA000C94D2018091BA008F7D64
:1003A0008093BA0040919E0000917D00041710F0E8
:1003B0000C94E1018091BA0088608093BA000C949B
:1003C000E6018091BA00877F8093BA0040919F0038
:1003D00000917D00041710F00C94F5018091B90094
:1003E00081608093B9000C94FA018091B9008E7FEE
:1003F0008093B9004091A00000917D00041710F097
:100400000C9409028091B90082608093B9000C9429
:100410000E028091B9008D7F8093B9004091A100B8
:1004200000917D00041710F00C941D028091BA0019
:1004300080648093BA000C9422028091BA008F7B72
:100440008093BA004091A20000917D00041710F043
:100450000C9431028091B90088608093B9000C94AB
:1004600036028091B900877F8093B9004091A30044
:1004700000917D00041710F00C9445028091B900A2
:1004800080618093B9000C944A028091B9008F7EFC
:100490008093B9004091A40000917D00041710F0F2
:1004A0000C9459028091B90084608093B9000C9437
:1004B0005E028091B9008B7F8093B9004091A500C6
:1004C00000917D00041710F00C946D028091B9002A
:1004D00080648093B9000C9472028091B9008F7B84
:1004E0008093B9004091A60000917D00041710F0A0
:1004F0000C9481028091B90080688093B9000C94BB
:1005000086028091B9008F778093B9004091A7004F
:1005100000917D00041710F00C9495028091B900B1
:1005200080628093B9000C949A028091B9008F7D0B
:100530008093B9004091A80000917D00041710F04D
:100540000C94A9028091BB0080648093BB000C9442
:10055000AE028091BB008F7B8093BB004091A900CD
:1005600000917D00041710F00C94BD028091BB0037
:1005700080628093BB000C94C2028091BB008F7D8F
:100580008093BB004091AA0000917D00041710F0F9
:100590000C94D1028091BB0080688093BB000C94C6
:1005A000D6028091BB008F778093BB004091AB0057
:1005B00000917D00041710F00C94E5028091BB00BF
:1005C00088608093BB000C94EA028091BB00877F17
:1005D0008093BB004091AC0000917D00041710F0A7
:1005E0000C94F9028091BB0084608093BB000C9452
:1005F000FE028091BB008B7F8093BB004091AD00D9
:1006000000917D00041710F00C940D038091BB0045
:1006100080618093BB000C9412038091BB008F7E9D
:100620008093BB004091AE0000917D00041710F054
:100630000C9421038091BB0081608093BB000C94DB
:1006400026038091BB008E7F8093BB004091AF005A
:1006500000917D00041710F00C9435038091B400D4
:1006600080648093B4000C943A038091B4008F7B33
:100670008093B4004091B00000917D00041710F009
:100680000C9449038091BB0082608093BB000C9462
:100690004E038091BB008D7F8093BB00A9EBB0E03F
:1006A0008C918BBBAAEBB0E08C9188BBABEBB0E03C
:1006B0008C9185BBA4EBB0E08C9186FBA2E3B0E00B
:1006C0008C9187F98C938F918FBFFF91EF91DF9180
:1006D000CF91BF91AF919F918F917F916F915F91DA
:1006E0004F913F912F911F910F91BF90AF907F90AD
:1006F0005F904F903F902F901F900F9018958BB761
:100700008F7B8BBF78940E94F903A8EBB0E02C9309
:10071000A7EBB0E01C93A7EBB0E08C918F778C93A4
:100720008091B40080688093B40018958F939F9354
:100730008FB73395539509F4439591E892BF9F91F4
:100740008FBF8F91189580917C00882309F081E0FC
:10075000089580917C00882309F408950F929F9357
:10076000AF93BF937F9380917C008823E1F3F8944B
:1007700080917C008A9580937C0090917A00A0E61D
:10078000B0E0A90F0024B01D8C9193959A3109F423
:10079000992790937A0078947F91BF91AF919F9120
:1007A0000F9008958D9103D03A95E1F708955D9BE0
:1007B000FECF8CB9089588EE93E00CD03197D9F72D
:1007C00008953197F1F70895689462F80895E894D0
:1007D00062F80895EF93FF93EE27E82BE92B31F0B1
:1007E000E0EAFFE03197F1F70197D1F7FF91EF9140
:1007F00008950F933F934F935F932F923F928F9360
:100800009F938FB78F9383B78F93826083BF89B78E
:100810008F93816089BF81E882BF552744273327A2
:10082000483008F047C0373324F4829BF8CFF8CF24
:1008300041C04830ECF78299FCCF33273232D4F5EF
:10084000829BFCCF932F332711272227913110F061
:10085000969511E0292E2694322C290E990F390EE7
:10086000113021F0321534F58299FCCF33270CE09A
:100870003215F0F3829909C08894111F221F331595
:10088000CCF4829BFCCF332708C00894111F221F91
:10089000331584F48299FCCF33270A9549F7912FB9
:1008A000991F221F991F221F25FB17F926FB16F9F6
:1008B0002F7102C01FEF2FEF8F9189BF8F9183BFE0
:1008C0008F918FBF9F918F913F902F905F914F910C
:1008D0003F910F9108957F930F93AF93BF938F93A1
:1008E0009F938FB78F9380917C000AE1081B21F4BE
:1008F0009CB10E94E40312C000917B00A0E6B0E02E
:1009000077279CB1A00FB71F9C93839580937C00A1
:1009100003950A3109F4002700937B008F918FBF64
:100920009F918F91BF91AF910F917F911895FF93F8
:10093000881BF9E0001FFA9511F4FF910895881FB4
:0E094000841B18F4840F8894F5CF0894F3CF2D
:00000001FF
